:1000000012C02CC02BC02AC0D7C328C027C026C00E
:1000100025C064C223C022C021C020C03DC01EC074
:100020001DC01CC01BC011241FBECFE5D4E0DEBF25
:10003000CDBF10E0A0E6B0E0ECE9F0E102C0059031
:100040000D92AC3AB107D9F710E0ACEAB0E001C0CC
:100050001D92AF3DB107E1F720D41EC8D1CF882350
:1000600031F090E00F920F909F5F9817D8F30895AA
:100070000F931F93082F882361F010E08AEFEFDFC2
:100080008AEFEDDF8AEFEBDF8AEFE9DF1F5F101702
:10009000A8F31F910F9108951F920F920FB60F9220
:1000A00011248F939F9384B195B19093CE00809348
:1000B000CD009F918F910F900FBE0F901F901895BC
:1000C000806487B98AE0CBDFE5E5F0E080E98083F2
:1000D000889580818F7780832091CD003091CE00EC
:1000E000822F932F0895EF92FF920F931F93CF9338
:1000F000DF93EC017B01D9018881998182179307F5
:1001000020F0FB016081718168C0BA01660F771F22
:10011000FE01E60FF71F808191812817390730F023
:10012000F701E60FF71F6081718157C000E01FC023
:10013000C901860F971F95958795282F90E0BC01E0
:10014000660F771FFE01E60FF71F0190F081E02D8B
:10015000AE17BF0710F4422F0AC0EA17FB0730F0B2
:10016000F701E60FF71F6081718137C0022F602F02
:1001700070E0242F30E0CB01019682179307C4F280
:10018000A901440F551FCB01880F991FF701E80FF4
:10019000F91F00811181F701E40FF51F20813181E2
:1001A000201B310BFE01E80FF91F80819181A81BF4
:1001B000B90BFE01E40FF51F60817181681B790B9B
:1001C000A29FC001A39F900DB29F900D1124EED667
:1001D000862F972FBC01600F711F862F972FDF91FD
:1001E000CF911F910F91FF90EF900895E5E3F0E01C
:1001F00080818D7F80838081846080830895E5E3A2
:10020000F0E080818260808380818B7F808308958D
:100210000F931F9308E310E0F801808182608083D0
:1002200080E526DFF80180818D7F80831F910F910B
:100230000895FF920F931F93CF93DF938091D30084
:100240009091D400892B09F043C1B69B06C08091E0
:10025000DE00882311F01092DE0086B3882334F488
:100260008091C700882311F01092C700B59B06C08B
:100270008091B800882311F01092B800B49B06C09A
:100280008091D500882311F01092D500B39B06C051
:100290008091AD00882311F01092AD00B69910C086
:1002A0008091DE00882309F4B3DF84E6E1DE81E09B
:1002B00090E09093D4008093D30081E08093DE009F
:1002C00086B3882384F08091C700882309F4A0DFD7
:1002D00084E6CEDE82E090E09093D4008093D30059
:1002E00081E08093C700B59944C08091B80088230D
:1002F00009F03FC08DDF1092B1001092B000B599A7
:1003000026C08091B0009091B100889700F5FF243D
:10031000F39400ED17E0C6E3D0E082E3A9DEF092AB
:10032000D7001093700000936F008091B0009091FF
:10033000B10001969093B1008093B000888185FD53
:1003400006C08091B0009091B100889730F3B599C4
:100350000AC086E090E09093D4008093D30081E0BF
:100360008093B80006C083E090E09093D40080931F
:10037000D300B49944C08091D500882309F03FC0D0
:1003800047DF1092B1001092B000B49926C080915E
:10039000B0009091B100889700F5FF24F39400ED30
:1003A00017E0C6E3D0E082E363DEF092D70010935B
:1003B000700000936F008091B0009091B1000196A1
:1003C0009093B1008093B000888184FD06C0809135
:1003D000B0009091B100889730F3B4990AC087E0DB
:1003E00090E09093D4008093D30081E08093D50077
:1003F00006C084E090E09093D4008093D300B3993A
:1004000044C08091AD00882309F03FC001DF109205
:10041000B1001092B000B39926C08091B0009091C5
:10042000B100889700F5FF24F39400ED17E0C6E3D0
:10043000D0E082E31DDEF092D700109370000093AD
:100440006F008091B0009091B10001969093B1003F
:100450008093B000888183FD06C08091B0009091A8
:10046000B100889730F3B3990AC088E090E0909388
:10047000D4008093D30081E08093AD0006C085E076
:1004800090E09093D4008093D3008091D30090911A
:10049000D400892BE9F080ED97E090937000809371
:1004A0006F0081E08093D7001092CA001092C900BB
:1004B0001092D2001092D1008091D600813041F488
:1004C0008091D3009091D400029711F41092D6003D
:1004D000DF91CF911F910F91FF9008951F920F927E
:1004E0000FB60F9211242F933F934F935F936F9307
:1004F0007F938F939F93AF93BF93EF93FF9382EB81
:1005000082BF80916D0090916E00019790936E0074
:1005100080936D0080916D0090916E00892BC1F4E5
:100520008091AC00882321F481E08093AC0002C06C
:100530001092AC0084E190E090936E0080936D0087
:100540008091BE009091BF009093CC008093CB002F
:100550008091D600882309F040C08091D10090910D
:10056000D20001969093D2008093D100805797419A
:1005700069F48091C9009091CA0001969093CA00D5
:100580008093C9001092D2001092D1008091BE00D9
:100590009091BF008059914030F08091C9009091B6
:1005A000CA000F9769F08091BE009091BF008059FA
:1005B000914098F48091C9009091CA00CC9769F459
:1005C00081E08093D6001092D2001092D100109258
:1005D000CA001092C9008093BD002091BE003091E6
:1005E000BF008091B4009091B500A091B600B09189
:1005F000B70040E050E00397A109B10982179307C3
:10060000A407B50774F52091BE003091BF0080911A
:10061000B4009091B500A091B600B091B70040E051
:1006200050E00396A11DB11D281739074A075B0743
:10063000C4F48091B2009091B30001979093B300FD
:100640008093B200892BA9F48091C800882389F493
:100650008091D600882369F4DBDD81E08093C800B7
:1006600008C01092C8008EE591E09093B30080938B
:10067000B20080917500909176000197909376007A
:1006800080937500FF91EF91BF91AF919F918F91F2
:100690007F916F915F914F913F912F910F900FBE7E
:1006A0000F901F901895E2ECF0E01182108280818B
:1006B00091813297918380838091CF009091D00077
:1006C00084369105C0F0E0ECF0E08091CF0090918D
:1006D000D000845690409093D0008093CF008081CA
:1006E00091810196918380838091CF009091D00079
:1006F0008436910550F78091CF009091D0000A97F1
:10070000B0F0E2ECF0E08091CF009091D0000A9739
:100710009093D0008093CF00808191810196918346
:1007200080838091CF009091D0000A9760F78091EC
:10073000CF009091D0009093C5008093C40008959D
:1007400012BAE5E3F0E08081886380838091D6006F
:10075000813049F4E091AE00F091AF00E659FF4FCF
:10076000808182BB0FC0E091AE00F091AF00EE0F30
:10077000FF1FE054FF4F0190F081E02DE05AFF4F42
:10078000808182BB8091C6008823A9F4E5E3F0E074
:1007900040818091AE009091AF0025E030E0281BB1
:1007A000390B81E090E002C0880F991F2A95E2F78B
:1007B00080958423808308951F920F920FB60F9225
:1007C00011242F933F934F935F936F937F938F9356
:1007D0009F93AF93BF93EF93FF9383E884BD809182
:1007E000D700813061F58091B4009091B500A0915F
:1007F000B600B091B7009093D0008093CF00809165
:100800006F00909170009C01215030403093700037
:1008100020936F008091AC00882351F48091C60032
:10082000882321F481E08093C60002C01092C600A4
:10083000232B69F41092C6001092D70008C0809153
:10084000CB009091CC009093D0008093CF002BDF11
:1008500077DF8091AE009091AF0001969093AF004A
:100860008093AE008091AE009091AF00039720F08E
:100870001092AF001092AE00FF91EF91BF91AF9137
:100880009F918F917F916F915F914F913F912F91A8
:100890000F900FBE0F901F9018952F923F924F927E
:1008A0005F926F927F928F929F92AF92BF92CF9200
:1008B000DF92EF92FF920F931F93CF93DF938CEF12
:1008C00088BB93E097BB30E435BB8EE384BB8FEFEE
:1008D00082BB81BB85E083BF82EB82BF23E82FBD53
:1008E0009EBD1DBC1CBC17BC16BC1BBC1ABC19BCD5
:1008F00018BC12BC84E085BD24BD13BC15BE81E4C8
:1009000089BF80E888B910BE37B98EE886B980E023
:1009100090E09DD38233910518F0815E914080F084
:1009200000E010E0C8016AEF70E096D3C8010296BB
:100930006CE271E091D3C80104966EE571E08CD34E
:100940000F2EF0E0EF2EF0E0FF2EF02DC7017FD349
:100950000F2EF8EDCF2EF0E0DF2EF02DD601119600
:100960009C938E9312968D01C701029670D3F80165
:1009700091838083C70104966AD3F60134969183EC
:100980008083D6018D919C91A0E0B0E08093B4006B
:100990009093B500A093B600B093B70081E0809328
:1009A000D60078940F2EF7E72F2EF0E03F2EF02D93
:1009B000C5E3D0E00F2EFFEF4F2EF3E05F2EF0E007
:1009C0006F2EF0E07F2EF02D0F2EFBE4AF2EBB2418
:1009D000F02D0F2EFAE48F2E9924F02D80E070DB9D
:1009E0009093CE008093CD002091CD003091CE0029
:1009F000C10161E970E04CE050E075DB9093BF000D
:100A00008093BE00809175009091760018161906AB
:100A10000CF411C12091BE003091BF008091B40050
:100A20009091B500A091B600B091B70040E050E0C1
:100A30000897A109B10982179307A407B5070CF01D
:100A400090C02091BE003091BF008091B400909181
:100A5000B500A091B600B091B70040E050E0049618
:100A6000A11DB11D281739074A075B070CF079C093
:100A70008091BE009091BF002091B4003091B500EC
:100A80004091B6005091B700A0E0B0E08217930704
:100A9000A407B5079CF48091710090917200A09119
:100AA0007300B09174000196A11DB11D8093710077
:100AB00090937200A0937300B09374008091BE0075
:100AC0009091BF002091B4003091B5004091B600E4
:100AD0005091B700A0E0B0E0281739074A075B073C
:100AE0009CF48091710090917200A0917300B0917C
:100AF00074000197A109B10980937100909372006D
:100B0000A0937300B0937400809171009091720073
:100B1000A0917300B0917400BB2344F41092710053
:100B20001092720010927300109274008091710004
:100B300090917200A0917300B09174008050924027
:100B4000A040B0400CF471C08FEF91E0A0E0B0E0A5
:100B50008093710090937200A0937300B09374001F
:100B600064C08091B4009091B500A091B600B0919E
:100B7000B70087399105A105B1050CF44AC0209151
:100B8000BE003091BF008091B4009091B500A0915B
:100B9000B600B091B70040E050E08497A109B109D8
:100BA00082179307A407B507A4F52091BE003091E2
:100BB000BF008091B4009091B500A091B600B091B3
:100BC000B70040E050E08496A11DB11D28173907F9
:100BD0004A075B07F4F46091B4007091B50080910E
:100BE000B6009091B700665970408040904022E076
:100BF00030E040E050E0EED1225E3F4F4F4F5F4F7C
:100C000020937100309372004093730050937400EE
:100C10000CC08EE190E0A0E0B0E080937100909372
:100C20007200A0937300B0937400A9E1B0E0B09398
:100C30007600A09375008091D600882309F057C0F4
:100C40006091B4007091B5008091B6009091B700AA
:100C5000E090BE00F090BF002091710030917200D2
:100C600040917300509174006E5F7F4F8F4F9F4F84
:100C700000E010E06E197F09800B910B78D1609332
:100C8000B9007093BA008093BB009093BC00209190
:100C9000BE003091BF008091B4009091B500A0914A
:100CA000B600B091B70040E050E00697A109B10945
:100CB00082179307A407B507C4F42091BE003091B2
:100CC000BF008091B4009091B500A091B600B091A2
:100CD000B70040E050E00696A11DB11D2817390766
:100CE0004A075B0714F482DA10C089DA0EC010924A
:100CF000B9001092BA001092BB001092BC0088811B
:100D0000826088838881846088838091B900909113
:100D1000BA00A091BB00B091BC0080509440A040AC
:100D2000B04044F04092B9005092BA006092BB00CB
:100D30007092BC008091B9009091BA00A091BB0064
:100D4000B091BC00BB2344F41092B9001092BA00D9
:100D50001092BB001092BC006CDA8091D30090918D
:100D6000D400019781F58091B4009091B500A091D5
:100D7000B600B091B7000596A11DB11D8093B400D7
:100D80009093B500A093B600B093B7008091B400E3
:100D90009091B500A091B600B091B700815E9140EE
:100DA000A040B04064F080EE91E0A0E0B0E080931D
:100DB000B4009093B500A093B600B093B700109222
:100DC000D4001092D3008091D3009091D400029768
:100DD00079F58091B4009091B500A091B600B091E2
:100DE000B7000597A109B1098093B4009093B500AD
:100DF000A093B600B093B7008091B4009091B50075
:100E0000A091B600B091B700C297A105B10564F4F6
:100E100082E390E0A0E0B0E08093B4009093B5004E
:100E2000A093B600B093B7001092D4001092D300F4
:100E30008091D3009091D400039718F18091D30052
:100E40009091D4000697E8F48091D3009091D4005B
:100E50000397880F991FF601E80FF91F8081918190
:100E6000A0E0B0E08093B4009093B500A093B600EA
:100E7000B093B70091E09093D7001092D4001092F5
:100E8000D3008091D3009091D400069708F444C019
:100E90008091D3009091D400099708F03DC0F89458
:100EA0008091D3009091D40006972091B4003091A6
:100EB000B5004091B6005091B700880F991FF60118
:100EC000E80FF91F318320832091D3003091D400A3
:100ED0008091D3009091D4000697880F991FF60156
:100EE000E80FF91F6081718126503040220F331FB7
:100EF00080E090E0820F931FAFD0789489D982E38D
:100F0000B7D886D982E3B4D883D9A1E0A093D7001B
:100F10001092D4001092D3008091BD00813061F412
:100F200077D982E3A5D874D982E3A2D871D982E3B4
:100F30009FD86ED91092BD008091B9009091BA00EF
:100F4000A091BB00B091BC00892F9A2FAB2FBB277B
:100F5000A7FDBA95F50180838091B9009091BA0000
:100F6000A091BB00B091BC00F401808337CD629F9B
:100F7000D001739FF001829FE00DF11D649FE00D91
:100F8000F11D929FF00D839FF00D749FF00D659FF2
:100F9000F00D9927729FB00DE11DF91F639FB00DF1
:100FA000E11DF91FBD01CF0111240895AA1BBB1B30
:100FB00051E107C0AA1FBB1FA617B70710F0A61B59
:100FC000B70B881F991F5A95A9F780959095BC017A
:100FD000CD01089597FB092E05260ED057FD04D0AC
:100FE00014D00AD0001C38F45095409530952195C6
:100FF0003F4F4F4F5F4F0895F6F79095809570954E
:1010000061957F4F8F4F9F4F0895A1E21A2EAA1B23
:10101000BB1BFD010DC0AA1FBB1FEE1FFF1FA217A8
:10102000B307E407F50720F0A21BB30BE40BF50BA5
:10103000661F771F881F991F1A9469F7609570952E
:10104000809590959B01AC01BD01CF010895A8E169
:10105000B0E042E050E005C012D0272F11C0DC0103
:10106000CB01FC01E199FECF06C0FFBBEEBBE09ACD
:1010700031960DB20D9241505040B8F70895262F89
:10108000E199FECF9FBB8EBB2DBB0FB6F894E29AC1
:0C109000E19A0FBE01960895F894FFCF7E
:10109C003F065B4F666D7D077F6F3F71710100D01E
:1010AC00071E000000F401EE0040014E015C0169D6
:1010BC0001740176018E019A01A501AD01C301E80D
:1010CC000128008000A200C200E100F900FF00111D
:0C10DC000135014A016601A401EA01008F
:00000001FF
